:100000000128831601308500003086000E309F00E5
:1000100070308F000030900083120030920005177E
:1000200085170230AA0002210611861006108611DB
:1000300005308820643064212B202B2020201C28B0
:10004000290807398207592838284728502867285F
:100050007D28622872283620AB003C30642136208F
:10006000A90A2B02053C03182B2808000030572949
:100070000430A82086153C3064210530A8200630C5
:10008000A8200730A82086110330882008000330FC
:1000900088208615503064210F30A8208611080072
:1000A000033088208615503064210E30A820861138
:1000B000080086153C3064210830A8200930A820AB
:1000C000861108000D30A8200D30A82008008615E4
:1000D0003C3064210130A8200230A8200330A82041
:1000E0008611080086153C3064211030A82011309C
:1000F000A8201230A8208611080086153C30642103
:100100000A30A8200B30A8200C30A8208611080047
:10011000AC008614902086109020AC0B8928080033
:1001200028306429A1001130061786139B2021086E
:100130009B2086170800A2000830AC00A20D031C0B
:1001400086120318861606130617AC0B9E280800A5
:100150000615AE200611323064210800B120D420EB
:100160000800FF3EA5000310A50D0310A50D0630E5
:10017000A507A601BC200800F020A0301021260809
:10018000102125081021F020A13010213021A300DA
:100190003F213021A4003F213021A7003F21302101
:1001A000A8004B2102210800F020A03010212408D3
:1001B000102123081021F020A1301021E0283F2138
:1001C00030219220A70BDF28A80BDF284B2102212A
:1001D0000800B000000000000000B00BEA28080092
:1001E00083160513831205130000831685178312E7
:1001F000000005178513831685138312000005136D
:100200002010080005138513831685138312000040
:1002100005170000831685178312000005130800D8
:10022000A1000830AC00A10D8513831603188517B3
:10023000031C85138312000005170000000005133E
:10024000AC0B1329831685178312000000000517D5
:100250000000851F2E29051320140800051308002F
:100260000830AC0083168517831205170310851B11
:1002700003140513A10DAC0B3529210808008513C3
:10028000831685138312000005170000000000008C
:100290000000051308008316851783120000000074
:1002A00005170000000000000000051308000339D6
:1002B000A1000310A10DA10DA10D210805389F007B
:1002C0001F1960291E080800B300B200B100B10B6D
:0C02D0006729B20B6629B30B65290800F2
:02400E00302F51
:00000001FF
